:02000000E229F3
:10000600000000008312031305150000000005110F
:020016000800E0
:100018008312031385150000000005150000000079
:0A002800851100000000051108001A
:0E0032008312031330088A002F088200080092
:10004000831203133108003A031D2928F930F00008
:1000500008003108013A031D3028C030F0000800C4
:100060003108023A031D3728B530F0000800310886
:10007000033A031D3E28E530F00008003108043A39
:10008000031D4528CC30F00008003108053A031D57
:100090004C286D30F00008003108063A031D532843
:1000A0007D30F00008003108073A031D5A28C1309E
:1000B000F00008003108083A031D6128FD30F00007
:1000C00008003108093A031D6828ED30F0000800E7
:0200D000080026
:1000D20083120313AE01831685158312A501250829
:1000E200083A03198328AE0D2E10000000000515F2
:1000F20085197D282E107E282E140000000005117F
:10010200A50A702803208316851183122E08F00099
:04011200F1010800EF
:10011600831203138511000000000515000000007E
:0801260085150000000008002F
:10012E0083120313B11B9D2885119E28851503206C
:10013E00311BA3288511A42885150320B11AA928DF
:10014E008511AA2885150320311AAF288511B028EC
:10015E0085150320B119B5288511B62885150320FC
:10016E003119BB288511BC2885150320B118C1286B
:10017E008511C228851503203118C7288511C82876
:0E018E008515032085150320000000000800E1
:10019C000C20D030B10097200230B10097202218EB
:1001AC00D9282E10DA282E14A218DE28AE10DF283B
:1001BC00AE142219E3282E11E4282E15A219E828D2
:1001CC00AE11E928AE152718ED282E12EE282E16A2
:1001DC00A718F228AE12F328AE162719F7282E13FB
:1001EC00F8282E17A719FC28AE13FD28AE172E08D9
:0801FC00B10097208B200800E0
:100204000C20D030B1009720B1019720B101972084
:1002140024180E292E100F292E14A4181329AE10F9
:100224001429AE14241918292E1119292E15A419CC
:100234001D29AE111E29AE15231822292E12232999
:100244002E16A3182729AE122829AE1623192C29F5
:100254002E132D292E17A3193129AE133229AE17C7
:0A0264002E08B10097208B2008003F
:10026E008312031320082606031D5429A0018316AA
:10027E00861606160630FD00FD0B4329000083127C
:10028E00861A4C29A20A0130A100061A5129A40A85
:10029E000230A1008316861206128312A00A0800ED
:1002AE0019208A110A128000840AAF0A0319B00AB3
:0802BE00F003031D572908009D
:1002C6000C20D030B10097200130B10097200C20CF
:1002D600D130B100972069207008A4008B20240833
:1002E600A300A30CA313A30CA313A30CA313A30C87
:1002F600A3132412A4122413A4130C20D030B1008B
:1003060097200230B10097200C20D130B100972001
:1003160069207008A2008B202208F000F00CF01370
:10032600F00CF013F00CF013F00CF0137008A700AB
:100336002212A2122213A2137008B1002020700804
:10034600AC002208B10020207008AB002308B100E1
:1003560020207008AA002408B10020207008AD00F3
:0203660008008D
:100368008312031322080A3A031DC229A20127088F
:10037800023A031DC129A701C229A70A2708023A80
:10038800031DCC292208043A031DCC29A701A20188
:100398002708033C0318D129A70122080A3C03189F
:1003A800D629A20124080A3A031DE129A401A30AB7
:0C03B8002308063A031DE129A3010800F8
:1003C40083120313A00107309F0050308100433093
:1003D400831681008B018501831205138513051093
:1003E4008510831686018312860105158515A810CC
:1003F4002810A0011230A600A901A101A701A201A1
:10040400A301A4010330FB008A30FC005530FD0039
:10041400FD0B0A2AFC0B0A2AFB0B0A2A0000000027
:100424006321851037212C0886000517B421053077
:10043400FC007930FD00FD0B1D2AFC0B1D2A000079
:10044400000005131030FD00FD0B262A00002B08C8
:100454008600A8182F2A8610302A861485172108AA
:10046400013A031D4C2AA101CE202708B100202007
:100474007008AC002208B10020207008AB000430E2
:10048400FC00A130FD00FD0B452AFC0B452A0000B1
:100494000000702A2108023A031D662AA1010221E4
:1004A4002308B10020207008AA002408B1002020ED
:1004B4007008AD000430FC008030FD00FD0B602AA4
:1004C400FC0B602A0000702A0530FC007930FD0026
:1004D400FD0B6A2AFC0B6A2A000000008513103009
:1004E400FD00FD0B732A00002A0886000514003065
:1004F400003A031D7F2A28302906031D922AA901E8
:100504000230A806A818882A6321912A0330FC0027
:100514000D30FD00FD0B8C2AFC0B8C2A00009C2A5C
:100524000330FC001030FD00FD0B962AFC0B962ACC
:1005340000000000A90A0330FC006730FD00FD0B39
:10054400A12AFC0BA12A000005101030FD00FD0BB0
:10055400A92A00002D08860085140530FC00793096
:10056400FD00FD0BB32AFC0BB32A00000000132A84
:02057400BA2AA1
:02400E00182177
:00000001FF
